:1000000027C036C035C034C033C032C031C030C064
:100010002FC02EC02DC0DDC02BC02AC029C028C0D3
:1000200027C0000000000004030201000000003BA4
:1000300000380000003A0037000101010101010110
:1000400001020202010204081020408004020100A3
:1000500011241FBECFE5D1E0DEBFCDBF20E0A0E67A
:10006000B0E001C01D92AB36B207E1F7FCD061C130
:10007000C7CF90E0FC01EC5BFF4F2491875C9F4F62
:10008000FC018491882399F090E0880F991FFC016E
:10009000ED5CFF4FA591B491FC01E35DFF4F8591AD
:1000A00094918FB7F894EC91E22BEC938FBF089565
:1000B00090E0FC01EE5DFF4F3491FC01EC5BFF4FE3
:1000C0002491FC01E75CFF4FE491EE23B9F0332368
:1000D00029F0323019F198F43130E1F0F0E0EE0F10
:1000E000FF1FE35DFF4FA591B4918FB7F894EC919A
:1000F000611117C020952E232C938FBF08953330A4
:1001000029F0343059F78FB58F7D02C08FB58F77C6
:100110008FBDE4CF80B78F7780BFE0CF80B78F7D72
:10012000FBCF2E2BE9CF3FB7F894809165009091DB
:100130006600A0916700B091680022B708B600FE83
:1001400005C02F3F19F00196A11DB11D3FBFBA2F69
:10015000A92F982F8827BC01CD01620F711D811D29
:10016000911D46E0660F771F881F991F4A95D1F7AA
:1001700008958F929F92AF92BF92CF92DF92EF92AB
:10018000FF924B015C01CFDF6B017C01CCDF6C196E
:100190007D098E099F09683E734081059105B0F382
:1001A00021E0821A9108A108B10888EEC80E83E008
:1001B000D81EE11CF11C81149104A104B10431F793
:1001C000FF90EF90DF90CF90BF90AF909F908F9077
:1001D00008951F920F920FB60F9211242F933F9301
:1001E0008F939F93AF93BF93809161009091620032
:1001F000A0916300B09164003091600020E3230F70
:100200002D3758F54096A11DB11D209360008093B5
:10021000610090936200A0936300B09364008091AA
:10022000650090916600A0916700B091680001960A
:10023000A11DB11D8093650090936600A093670097
:10024000B0936800BF91AF919F918F913F912F9193
:100250000F900FBE0F901F90189523EB230F419620
:10026000A11DB11DD2CF789480B7826080BF80B7C6
:10027000816080BF83B7826083BF83B7816083BFA3
:1002800089B7816089BF1EBC8EB582608EBD8FB577
:1002900081608FBD3298319A309A379A83E0E9DED7
:1002A00087E0E7DE88E0E5DE12E080E0E82E80E02F
:1002B000F82E64E670E080E090E05BDF1D9817B9EF
:1002C000369A3699FECF84B1C5B1DC2FC82FD093B2
:1002D0006A00C0936900C73682E0D8074CF060E03E
:1002E00083E0E6DE60E087E0E3DE61E088E0E0DE18
:1002F000CE01825C9140843A910598F460E083E0FD
:10030000D7DE61E087E0D4DE60E088E0D1DE64EF34
:1003100071E080E090E02DDFE114F10451F270DE35
:10032000C8CFC23CD1409CF761E083E0C1DE60E011
:06033000E9CFF894FFCFB5
:00000001FF
